ARM GAS  C:\Users\varun\AppData\Local\Temp\ccU3kTLK.s 			page 1


   1              		.syntax unified
   2              		.cpu cortex-m0plus
   3              		.fpu softvfp
   4              		.eabi_attribute 20, 1
   5              		.eabi_attribute 21, 1
   6              		.eabi_attribute 23, 3
   7              		.eabi_attribute 24, 1
   8              		.eabi_attribute 25, 1
   9              		.eabi_attribute 26, 1
  10              		.eabi_attribute 30, 1
  11              		.eabi_attribute 34, 0
  12              		.eabi_attribute 18, 4
  13              		.thumb
  14              		.syntax unified
  15              		.file	"main.c"
  16              		.text
  17              	.Ltext0:
  18              		.cfi_sections	.debug_frame
  19              		.section	.text.LCD_Disp,"ax",%progbits
  20              		.align	2
  21              		.global	LCD_Disp
  22              		.code	16
  23              		.thumb_func
  24              		.type	LCD_Disp, %function
  25              	LCD_Disp:
  26              	.LFB34:
  27              		.file 1 "main.c"
   1:main.c        **** /* ========================================
   2:main.c        ****  *
   3:main.c        ****  * Copyright YOUR COMPANY, THE YEAR
   4:main.c        ****  * All Rights Reserved
   5:main.c        ****  * UNPUBLISHED, LICENSED SOFTWARE.
   6:main.c        ****  *
   7:main.c        ****  * CONFIDENTIAL AND PROPRIETARY INFORMATION
   8:main.c        ****  * WHICH IS THE PROPERTY OF your company.
   9:main.c        ****  *
  10:main.c        ****  * ========================================
  11:main.c        **** */
  12:main.c        **** #include "project.h"
  13:main.c        **** void LCD_Disp(void);
  14:main.c        **** void main_board(void);
  15:main.c        **** void extension_board(void);
  16:main.c        **** void Extension_1(void);
  17:main.c        **** 
  18:main.c        **** int main(void)
  19:main.c        **** {
  20:main.c        ****     CyGlobalIntEnable; /* Enable global interrupts. */
  21:main.c        **** 
  22:main.c        ****     /* Place your initialization/startup code here (e.g. MyInst_Start()) */
  23:main.c        ****     LCD_Start();
  24:main.c        ****     CyDelay(10);
  25:main.c        ****     for(;;)
  26:main.c        ****     {
  27:main.c        ****         /* Place your application code here. */
  28:main.c        ****         if((HW_Select1_Read()==0) && (HW_Select2_Read()==0))
  29:main.c        ****         {
  30:main.c        ****             main_board();
ARM GAS  C:\Users\varun\AppData\Local\Temp\ccU3kTLK.s 			page 2


  31:main.c        ****         }
  32:main.c        ****         
  33:main.c        ****         if((HW_Select1_Read()==1) && (HW_Select2_Read()==0))
  34:main.c        ****         {
  35:main.c        ****             Extension_1();
  36:main.c        ****         }
  37:main.c        ****         if((HW_Select1_Read()==0) && (HW_Select2_Read()==1))
  38:main.c        ****         {
  39:main.c        ****             main_board();
  40:main.c        ****         }
  41:main.c        ****         
  42:main.c        ****     }
  43:main.c        **** }
  44:main.c        **** 
  45:main.c        **** void LCD_Disp(void)
  46:main.c        **** {
  28              		.loc 1 46 0
  29              		.cfi_startproc
  30              		@ args = 0, pretend = 0, frame = 0
  31              		@ frame_needed = 0, uses_anonymous_args = 0
  32 0000 10B5     		push	{r4, lr}
  33              		.cfi_def_cfa_offset 8
  34              		.cfi_offset 4, -8
  35              		.cfi_offset 14, -4
  47:main.c        ****    LCD_Position(0,3);
  36              		.loc 1 47 0
  37 0002 0321     		movs	r1, #3
  38 0004 0020     		movs	r0, #0
  39 0006 FFF7FEFF 		bl	LCD_Position
  40              	.LVL0:
  48:main.c        ****    LCD_PrintString("Smart_Box");
  41              		.loc 1 48 0
  42 000a 0848     		ldr	r0, .L2
  43 000c FFF7FEFF 		bl	LCD_PrintString
  44              	.LVL1:
  49:main.c        ****    CyDelay(100);
  45              		.loc 1 49 0
  46 0010 6420     		movs	r0, #100
  47 0012 FFF7FEFF 		bl	CyDelay
  48              	.LVL2:
  50:main.c        ****    LCD_Position(1,3);
  49              		.loc 1 50 0
  50 0016 0321     		movs	r1, #3
  51 0018 0120     		movs	r0, #1
  52 001a FFF7FEFF 		bl	LCD_Position
  53              	.LVL3:
  51:main.c        ****    LCD_PrintString("Testing");
  54              		.loc 1 51 0
  55 001e 0448     		ldr	r0, .L2+4
  56 0020 FFF7FEFF 		bl	LCD_PrintString
  57              	.LVL4:
  52:main.c        ****    CyDelay(100);
  58              		.loc 1 52 0
  59 0024 6420     		movs	r0, #100
  60 0026 FFF7FEFF 		bl	CyDelay
  61              	.LVL5:
  53:main.c        **** }
ARM GAS  C:\Users\varun\AppData\Local\Temp\ccU3kTLK.s 			page 3


  62              		.loc 1 53 0
  63              		@ sp needed
  64 002a 10BD     		pop	{r4, pc}
  65              	.L3:
  66              		.align	2
  67              	.L2:
  68 002c 00000000 		.word	.LC0
  69 0030 0C000000 		.word	.LC2
  70              		.cfi_endproc
  71              	.LFE34:
  72              		.size	LCD_Disp, .-LCD_Disp
  73              		.section	.text.main_board,"ax",%progbits
  74              		.align	2
  75              		.global	main_board
  76              		.code	16
  77              		.thumb_func
  78              		.type	main_board, %function
  79              	main_board:
  80              	.LFB35:
  54:main.c        **** 
  55:main.c        **** void main_board(void)
  56:main.c        **** {
  81              		.loc 1 56 0
  82              		.cfi_startproc
  83              		@ args = 0, pretend = 0, frame = 0
  84              		@ frame_needed = 0, uses_anonymous_args = 0
  85 0000 10B5     		push	{r4, lr}
  86              		.cfi_def_cfa_offset 8
  87              		.cfi_offset 4, -8
  88              		.cfi_offset 14, -4
  57:main.c        ****     Status_Write(1);
  89              		.loc 1 57 0
  90 0002 0120     		movs	r0, #1
  91 0004 FFF7FEFF 		bl	Status_Write
  92              	.LVL6:
  58:main.c        ****     CyDelay(100);
  93              		.loc 1 58 0
  94 0008 6420     		movs	r0, #100
  95 000a FFF7FEFF 		bl	CyDelay
  96              	.LVL7:
  59:main.c        ****     Status_Write(0);
  97              		.loc 1 59 0
  98 000e 0020     		movs	r0, #0
  99 0010 FFF7FEFF 		bl	Status_Write
 100              	.LVL8:
  60:main.c        ****     CyDelay(100);
 101              		.loc 1 60 0
 102 0014 6420     		movs	r0, #100
 103 0016 FFF7FEFF 		bl	CyDelay
 104              	.LVL9:
  61:main.c        **** 
  62:main.c        **** 
  63:main.c        ****     Router_Write(1);
 105              		.loc 1 63 0
 106 001a 0120     		movs	r0, #1
 107 001c FFF7FEFF 		bl	Router_Write
 108              	.LVL10:
ARM GAS  C:\Users\varun\AppData\Local\Temp\ccU3kTLK.s 			page 4


  64:main.c        ****     CyDelay(100);
 109              		.loc 1 64 0
 110 0020 6420     		movs	r0, #100
 111 0022 FFF7FEFF 		bl	CyDelay
 112              	.LVL11:
  65:main.c        ****     Router_Write(0);
 113              		.loc 1 65 0
 114 0026 0020     		movs	r0, #0
 115 0028 FFF7FEFF 		bl	Router_Write
 116              	.LVL12:
  66:main.c        ****     CyDelay(100);
 117              		.loc 1 66 0
 118 002c 6420     		movs	r0, #100
 119 002e FFF7FEFF 		bl	CyDelay
 120              	.LVL13:
  67:main.c        **** 
  68:main.c        ****     FAN_Write(1);
 121              		.loc 1 68 0
 122 0032 0120     		movs	r0, #1
 123 0034 FFF7FEFF 		bl	FAN_Write
 124              	.LVL14:
  69:main.c        ****     CyDelay(100);
 125              		.loc 1 69 0
 126 0038 6420     		movs	r0, #100
 127 003a FFF7FEFF 		bl	CyDelay
 128              	.LVL15:
  70:main.c        ****     FAN_Write(0);
 129              		.loc 1 70 0
 130 003e 0020     		movs	r0, #0
 131 0040 FFF7FEFF 		bl	FAN_Write
 132              	.LVL16:
  71:main.c        ****     CyDelay(100);
 133              		.loc 1 71 0
 134 0044 6420     		movs	r0, #100
 135 0046 FFF7FEFF 		bl	CyDelay
 136              	.LVL17:
  72:main.c        **** 
  73:main.c        ****     if(SIC_1_Read()!=0)
 137              		.loc 1 73 0
 138 004a FFF7FEFF 		bl	SIC_1_Read
 139              	.LVL18:
 140 004e 0028     		cmp	r0, #0
 141 0050 03D0     		beq	.L5
  74:main.c        ****     {
  75:main.c        ****        SOL_1_Write(0);
 142              		.loc 1 75 0
 143 0052 0020     		movs	r0, #0
 144 0054 FFF7FEFF 		bl	SOL_1_Write
 145              	.LVL19:
 146 0058 02E0     		b	.L6
 147              	.L5:
  76:main.c        ****     }
  77:main.c        ****     else
  78:main.c        ****     {
  79:main.c        ****        SOL_1_Write(1); 
 148              		.loc 1 79 0
 149 005a 0120     		movs	r0, #1
ARM GAS  C:\Users\varun\AppData\Local\Temp\ccU3kTLK.s 			page 5


 150 005c FFF7FEFF 		bl	SOL_1_Write
 151              	.LVL20:
 152              	.L6:
  80:main.c        ****     }
  81:main.c        ****     if(SIC_2_Read()!=0)
 153              		.loc 1 81 0
 154 0060 FFF7FEFF 		bl	SIC_2_Read
 155              	.LVL21:
 156 0064 0028     		cmp	r0, #0
 157 0066 03D0     		beq	.L7
  82:main.c        ****     {
  83:main.c        ****        SOL_2_Write(0);
 158              		.loc 1 83 0
 159 0068 0020     		movs	r0, #0
 160 006a FFF7FEFF 		bl	SOL_2_Write
 161              	.LVL22:
 162 006e 02E0     		b	.L8
 163              	.L7:
  84:main.c        ****     }
  85:main.c        ****     else
  86:main.c        ****     {
  87:main.c        ****        SOL_2_Write(1); 
 164              		.loc 1 87 0
 165 0070 0120     		movs	r0, #1
 166 0072 FFF7FEFF 		bl	SOL_2_Write
 167              	.LVL23:
 168              	.L8:
  88:main.c        ****     }
  89:main.c        ****     if(SIC_3_Read()!=0)
 169              		.loc 1 89 0
 170 0076 FFF7FEFF 		bl	SIC_3_Read
 171              	.LVL24:
 172 007a 0028     		cmp	r0, #0
 173 007c 03D0     		beq	.L9
  90:main.c        ****     {
  91:main.c        ****        SOL_3_Write(0);
 174              		.loc 1 91 0
 175 007e 0020     		movs	r0, #0
 176 0080 FFF7FEFF 		bl	SOL_3_Write
 177              	.LVL25:
 178 0084 02E0     		b	.L10
 179              	.L9:
  92:main.c        ****     }
  93:main.c        ****     else
  94:main.c        ****     {
  95:main.c        ****        SOL_3_Write(1); 
 180              		.loc 1 95 0
 181 0086 0120     		movs	r0, #1
 182 0088 FFF7FEFF 		bl	SOL_3_Write
 183              	.LVL26:
 184              	.L10:
  96:main.c        ****     }
  97:main.c        ****     if(SIC_4_Read()!=0)
 185              		.loc 1 97 0
 186 008c FFF7FEFF 		bl	SIC_4_Read
 187              	.LVL27:
 188 0090 0028     		cmp	r0, #0
ARM GAS  C:\Users\varun\AppData\Local\Temp\ccU3kTLK.s 			page 6


 189 0092 03D0     		beq	.L11
  98:main.c        ****     {
  99:main.c        ****        SOL_4_Write(0);
 190              		.loc 1 99 0
 191 0094 0020     		movs	r0, #0
 192 0096 FFF7FEFF 		bl	SOL_4_Write
 193              	.LVL28:
 194 009a 02E0     		b	.L12
 195              	.L11:
 100:main.c        ****     }
 101:main.c        ****     else
 102:main.c        ****     {
 103:main.c        ****        SOL_4_Write(1); 
 196              		.loc 1 103 0
 197 009c 0120     		movs	r0, #1
 198 009e FFF7FEFF 		bl	SOL_4_Write
 199              	.LVL29:
 200              	.L12:
 104:main.c        ****     }
 105:main.c        ****     if(SIC_5_Read()!=0)
 201              		.loc 1 105 0
 202 00a2 FFF7FEFF 		bl	SIC_5_Read
 203              	.LVL30:
 204 00a6 0028     		cmp	r0, #0
 205 00a8 03D0     		beq	.L13
 106:main.c        ****     {
 107:main.c        ****        SOL_5_Write(0);
 206              		.loc 1 107 0
 207 00aa 0020     		movs	r0, #0
 208 00ac FFF7FEFF 		bl	SOL_5_Write
 209              	.LVL31:
 210 00b0 02E0     		b	.L14
 211              	.L13:
 108:main.c        ****     }
 109:main.c        ****     else
 110:main.c        ****     {
 111:main.c        ****        SOL_5_Write(1); 
 212              		.loc 1 111 0
 213 00b2 0120     		movs	r0, #1
 214 00b4 FFF7FEFF 		bl	SOL_5_Write
 215              	.LVL32:
 216              	.L14:
 112:main.c        ****     }
 113:main.c        ****     if(SIC_6_Read()!=0)
 217              		.loc 1 113 0
 218 00b8 FFF7FEFF 		bl	SIC_6_Read
 219              	.LVL33:
 220 00bc 0028     		cmp	r0, #0
 221 00be 03D0     		beq	.L15
 114:main.c        ****     {
 115:main.c        ****        SOL_6_Write(0);
 222              		.loc 1 115 0
 223 00c0 0020     		movs	r0, #0
 224 00c2 FFF7FEFF 		bl	SOL_6_Write
 225              	.LVL34:
 226 00c6 02E0     		b	.L16
 227              	.L15:
ARM GAS  C:\Users\varun\AppData\Local\Temp\ccU3kTLK.s 			page 7


 116:main.c        ****     }
 117:main.c        ****     else
 118:main.c        ****     {
 119:main.c        ****        SOL_6_Write(1); 
 228              		.loc 1 119 0
 229 00c8 0120     		movs	r0, #1
 230 00ca FFF7FEFF 		bl	SOL_6_Write
 231              	.LVL35:
 232              	.L16:
 120:main.c        ****     }
 121:main.c        ****     if(SIC_7_Read()!=0)
 233              		.loc 1 121 0
 234 00ce FFF7FEFF 		bl	SIC_7_Read
 235              	.LVL36:
 236 00d2 0028     		cmp	r0, #0
 237 00d4 03D0     		beq	.L17
 122:main.c        ****     {
 123:main.c        ****        SOL_7_Write(0);
 238              		.loc 1 123 0
 239 00d6 0020     		movs	r0, #0
 240 00d8 FFF7FEFF 		bl	SOL_7_Write
 241              	.LVL37:
 242 00dc 02E0     		b	.L18
 243              	.L17:
 124:main.c        ****     }
 125:main.c        ****     else
 126:main.c        ****     {
 127:main.c        ****        SOL_7_Write(1); 
 244              		.loc 1 127 0
 245 00de 0120     		movs	r0, #1
 246 00e0 FFF7FEFF 		bl	SOL_7_Write
 247              	.LVL38:
 248              	.L18:
 128:main.c        ****     }
 129:main.c        ****     if(SIC_8_Read()!=0)
 249              		.loc 1 129 0
 250 00e4 FFF7FEFF 		bl	SIC_8_Read
 251              	.LVL39:
 252 00e8 0028     		cmp	r0, #0
 253 00ea 03D0     		beq	.L19
 130:main.c        ****     {
 131:main.c        ****        SOL_8_Write(0);
 254              		.loc 1 131 0
 255 00ec 0020     		movs	r0, #0
 256 00ee FFF7FEFF 		bl	SOL_8_Write
 257              	.LVL40:
 258 00f2 02E0     		b	.L20
 259              	.L19:
 132:main.c        ****     }
 133:main.c        ****     else
 134:main.c        ****     {
 135:main.c        ****        SOL_8_Write(1); 
 260              		.loc 1 135 0
 261 00f4 0120     		movs	r0, #1
 262 00f6 FFF7FEFF 		bl	SOL_8_Write
 263              	.LVL41:
 264              	.L20:
ARM GAS  C:\Users\varun\AppData\Local\Temp\ccU3kTLK.s 			page 8


 136:main.c        ****     }
 137:main.c        ****     LCD_Disp();
 265              		.loc 1 137 0
 266 00fa FFF7FEFF 		bl	LCD_Disp
 267              	.LVL42:
 138:main.c        **** }
 268              		.loc 1 138 0
 269              		@ sp needed
 270 00fe 10BD     		pop	{r4, pc}
 271              		.cfi_endproc
 272              	.LFE35:
 273              		.size	main_board, .-main_board
 274              		.section	.text.Extension_1,"ax",%progbits
 275              		.align	2
 276              		.global	Extension_1
 277              		.code	16
 278              		.thumb_func
 279              		.type	Extension_1, %function
 280              	Extension_1:
 281              	.LFB36:
 139:main.c        **** void Extension_1(void)
 140:main.c        **** {
 282              		.loc 1 140 0
 283              		.cfi_startproc
 284              		@ args = 0, pretend = 0, frame = 0
 285              		@ frame_needed = 0, uses_anonymous_args = 0
 286 0000 10B5     		push	{r4, lr}
 287              		.cfi_def_cfa_offset 8
 288              		.cfi_offset 4, -8
 289              		.cfi_offset 14, -4
 141:main.c        ****     Status_Write(1);
 290              		.loc 1 141 0
 291 0002 0120     		movs	r0, #1
 292 0004 FFF7FEFF 		bl	Status_Write
 293              	.LVL43:
 142:main.c        ****     CyDelay(100);
 294              		.loc 1 142 0
 295 0008 6420     		movs	r0, #100
 296 000a FFF7FEFF 		bl	CyDelay
 297              	.LVL44:
 143:main.c        ****     Status_Write(0);
 298              		.loc 1 143 0
 299 000e 0020     		movs	r0, #0
 300 0010 FFF7FEFF 		bl	Status_Write
 301              	.LVL45:
 144:main.c        ****     CyDelay(100);
 302              		.loc 1 144 0
 303 0014 6420     		movs	r0, #100
 304 0016 FFF7FEFF 		bl	CyDelay
 305              	.LVL46:
 145:main.c        **** 
 146:main.c        ****     if(SIC_1_Read()!=0)
 306              		.loc 1 146 0
 307 001a FFF7FEFF 		bl	SIC_1_Read
 308              	.LVL47:
 309 001e 0028     		cmp	r0, #0
 310 0020 03D0     		beq	.L22
ARM GAS  C:\Users\varun\AppData\Local\Temp\ccU3kTLK.s 			page 9


 147:main.c        ****     {
 148:main.c        ****        SOL_8_Write(0);
 311              		.loc 1 148 0
 312 0022 0020     		movs	r0, #0
 313 0024 FFF7FEFF 		bl	SOL_8_Write
 314              	.LVL48:
 315 0028 02E0     		b	.L23
 316              	.L22:
 149:main.c        ****     }
 150:main.c        ****     else
 151:main.c        ****     {
 152:main.c        ****        SOL_8_Write(1); 
 317              		.loc 1 152 0
 318 002a 0120     		movs	r0, #1
 319 002c FFF7FEFF 		bl	SOL_8_Write
 320              	.LVL49:
 321              	.L23:
 153:main.c        ****     }
 154:main.c        ****     if(SIC_2_Read()!=0)
 322              		.loc 1 154 0
 323 0030 FFF7FEFF 		bl	SIC_2_Read
 324              	.LVL50:
 325 0034 0028     		cmp	r0, #0
 326 0036 03D0     		beq	.L24
 155:main.c        ****     {
 156:main.c        ****        SOL_7_Write(0);
 327              		.loc 1 156 0
 328 0038 0020     		movs	r0, #0
 329 003a FFF7FEFF 		bl	SOL_7_Write
 330              	.LVL51:
 331 003e 02E0     		b	.L25
 332              	.L24:
 157:main.c        ****     }
 158:main.c        ****     else
 159:main.c        ****     {
 160:main.c        ****        SOL_7_Write(1); 
 333              		.loc 1 160 0
 334 0040 0120     		movs	r0, #1
 335 0042 FFF7FEFF 		bl	SOL_7_Write
 336              	.LVL52:
 337              	.L25:
 161:main.c        ****     }
 162:main.c        ****     if(SIC_3_Read()!=0)
 338              		.loc 1 162 0
 339 0046 FFF7FEFF 		bl	SIC_3_Read
 340              	.LVL53:
 341 004a 0028     		cmp	r0, #0
 342 004c 03D0     		beq	.L26
 163:main.c        ****     {
 164:main.c        ****        SOL_6_Write(0);
 343              		.loc 1 164 0
 344 004e 0020     		movs	r0, #0
 345 0050 FFF7FEFF 		bl	SOL_6_Write
 346              	.LVL54:
 347 0054 02E0     		b	.L27
 348              	.L26:
 165:main.c        ****     }
ARM GAS  C:\Users\varun\AppData\Local\Temp\ccU3kTLK.s 			page 10


 166:main.c        ****     else
 167:main.c        ****     {
 168:main.c        ****        SOL_6_Write(1); 
 349              		.loc 1 168 0
 350 0056 0120     		movs	r0, #1
 351 0058 FFF7FEFF 		bl	SOL_6_Write
 352              	.LVL55:
 353              	.L27:
 169:main.c        ****     }
 170:main.c        ****     if(SIC_4_Read()!=0)
 354              		.loc 1 170 0
 355 005c FFF7FEFF 		bl	SIC_4_Read
 356              	.LVL56:
 357 0060 0028     		cmp	r0, #0
 358 0062 03D0     		beq	.L28
 171:main.c        ****     {
 172:main.c        ****        SOL_5_Write(0);
 359              		.loc 1 172 0
 360 0064 0020     		movs	r0, #0
 361 0066 FFF7FEFF 		bl	SOL_5_Write
 362              	.LVL57:
 363 006a 02E0     		b	.L29
 364              	.L28:
 173:main.c        ****     }
 174:main.c        ****     else
 175:main.c        ****     {
 176:main.c        ****        SOL_5_Write(1); 
 365              		.loc 1 176 0
 366 006c 0120     		movs	r0, #1
 367 006e FFF7FEFF 		bl	SOL_5_Write
 368              	.LVL58:
 369              	.L29:
 177:main.c        ****     }
 178:main.c        ****     if(SIC_5_Read()!=0)
 370              		.loc 1 178 0
 371 0072 FFF7FEFF 		bl	SIC_5_Read
 372              	.LVL59:
 373 0076 0028     		cmp	r0, #0
 374 0078 03D0     		beq	.L30
 179:main.c        ****     {
 180:main.c        ****        SOL_4_Write(0);
 375              		.loc 1 180 0
 376 007a 0020     		movs	r0, #0
 377 007c FFF7FEFF 		bl	SOL_4_Write
 378              	.LVL60:
 379 0080 02E0     		b	.L31
 380              	.L30:
 181:main.c        ****     }
 182:main.c        ****     else
 183:main.c        ****     {
 184:main.c        ****        SOL_4_Write(1); 
 381              		.loc 1 184 0
 382 0082 0120     		movs	r0, #1
 383 0084 FFF7FEFF 		bl	SOL_4_Write
 384              	.LVL61:
 385              	.L31:
 185:main.c        ****     }
ARM GAS  C:\Users\varun\AppData\Local\Temp\ccU3kTLK.s 			page 11


 186:main.c        ****     if(SIC_6_Read()!=0)
 386              		.loc 1 186 0
 387 0088 FFF7FEFF 		bl	SIC_6_Read
 388              	.LVL62:
 389 008c 0028     		cmp	r0, #0
 390 008e 03D0     		beq	.L32
 187:main.c        ****     {
 188:main.c        ****        SOL_3_Write(0);
 391              		.loc 1 188 0
 392 0090 0020     		movs	r0, #0
 393 0092 FFF7FEFF 		bl	SOL_3_Write
 394              	.LVL63:
 395 0096 02E0     		b	.L33
 396              	.L32:
 189:main.c        ****     }
 190:main.c        ****     else
 191:main.c        ****     {
 192:main.c        ****        SOL_3_Write(1); 
 397              		.loc 1 192 0
 398 0098 0120     		movs	r0, #1
 399 009a FFF7FEFF 		bl	SOL_3_Write
 400              	.LVL64:
 401              	.L33:
 193:main.c        ****     }
 194:main.c        ****     if(SIC_7_Read()!=0)
 402              		.loc 1 194 0
 403 009e FFF7FEFF 		bl	SIC_7_Read
 404              	.LVL65:
 405 00a2 0028     		cmp	r0, #0
 406 00a4 03D0     		beq	.L34
 195:main.c        ****     {
 196:main.c        ****        SOL_2_Write(0);
 407              		.loc 1 196 0
 408 00a6 0020     		movs	r0, #0
 409 00a8 FFF7FEFF 		bl	SOL_2_Write
 410              	.LVL66:
 411 00ac 02E0     		b	.L35
 412              	.L34:
 197:main.c        ****     }
 198:main.c        ****     else
 199:main.c        ****     {
 200:main.c        ****        SOL_2_Write(1); 
 413              		.loc 1 200 0
 414 00ae 0120     		movs	r0, #1
 415 00b0 FFF7FEFF 		bl	SOL_2_Write
 416              	.LVL67:
 417              	.L35:
 201:main.c        ****     }
 202:main.c        ****     if(SIC_8_Read()!=0)
 418              		.loc 1 202 0
 419 00b4 FFF7FEFF 		bl	SIC_8_Read
 420              	.LVL68:
 421 00b8 0028     		cmp	r0, #0
 422 00ba 03D0     		beq	.L36
 203:main.c        ****     {
 204:main.c        ****        SOL_1_Write(0);
 423              		.loc 1 204 0
ARM GAS  C:\Users\varun\AppData\Local\Temp\ccU3kTLK.s 			page 12


 424 00bc 0020     		movs	r0, #0
 425 00be FFF7FEFF 		bl	SOL_1_Write
 426              	.LVL69:
 427 00c2 02E0     		b	.L21
 428              	.L36:
 205:main.c        ****     }
 206:main.c        ****     else
 207:main.c        ****     {
 208:main.c        ****        SOL_1_Write(1); 
 429              		.loc 1 208 0
 430 00c4 0120     		movs	r0, #1
 431 00c6 FFF7FEFF 		bl	SOL_1_Write
 432              	.LVL70:
 433              	.L21:
 209:main.c        ****     }
 210:main.c        **** }
 434              		.loc 1 210 0
 435              		@ sp needed
 436 00ca 10BD     		pop	{r4, pc}
 437              		.cfi_endproc
 438              	.LFE36:
 439              		.size	Extension_1, .-Extension_1
 440              		.section	.text.main,"ax",%progbits
 441              		.align	2
 442              		.global	main
 443              		.code	16
 444              		.thumb_func
 445              		.type	main, %function
 446              	main:
 447              	.LFB33:
  19:main.c        ****     CyGlobalIntEnable; /* Enable global interrupts. */
 448              		.loc 1 19 0
 449              		.cfi_startproc
 450              		@ Volatile: function does not return.
 451              		@ args = 0, pretend = 0, frame = 0
 452              		@ frame_needed = 0, uses_anonymous_args = 0
 453 0000 10B5     		push	{r4, lr}
 454              		.cfi_def_cfa_offset 8
 455              		.cfi_offset 4, -8
 456              		.cfi_offset 14, -4
  20:main.c        **** 
 457              		.loc 1 20 0
 458              		.syntax divided
 459              	@ 20 "main.c" 1
 460 0002 62B6     		CPSIE   i
 461              	@ 0 "" 2
  23:main.c        ****     CyDelay(10);
 462              		.loc 1 23 0
 463              		.thumb
 464              		.syntax unified
 465 0004 FFF7FEFF 		bl	LCD_Start
 466              	.LVL71:
  24:main.c        ****     for(;;)
 467              		.loc 1 24 0
 468 0008 0A20     		movs	r0, #10
 469 000a FFF7FEFF 		bl	CyDelay
 470              	.LVL72:
ARM GAS  C:\Users\varun\AppData\Local\Temp\ccU3kTLK.s 			page 13


 471              	.L41:
  28:main.c        ****         {
 472              		.loc 1 28 0
 473 000e FFF7FEFF 		bl	HW_Select1_Read
 474              	.LVL73:
 475 0012 0028     		cmp	r0, #0
 476 0014 05D1     		bne	.L39
  28:main.c        ****         {
 477              		.loc 1 28 0 is_stmt 0 discriminator 1
 478 0016 FFF7FEFF 		bl	HW_Select2_Read
 479              	.LVL74:
 480 001a 0028     		cmp	r0, #0
 481 001c 01D1     		bne	.L39
  30:main.c        ****         }
 482              		.loc 1 30 0 is_stmt 1
 483 001e FFF7FEFF 		bl	main_board
 484              	.LVL75:
 485              	.L39:
  33:main.c        ****         {
 486              		.loc 1 33 0
 487 0022 FFF7FEFF 		bl	HW_Select1_Read
 488              	.LVL76:
 489 0026 0128     		cmp	r0, #1
 490 0028 05D1     		bne	.L40
  33:main.c        ****         {
 491              		.loc 1 33 0 is_stmt 0 discriminator 1
 492 002a FFF7FEFF 		bl	HW_Select2_Read
 493              	.LVL77:
 494 002e 0028     		cmp	r0, #0
 495 0030 01D1     		bne	.L40
  35:main.c        ****         }
 496              		.loc 1 35 0 is_stmt 1
 497 0032 FFF7FEFF 		bl	Extension_1
 498              	.LVL78:
 499              	.L40:
  37:main.c        ****         {
 500              		.loc 1 37 0
 501 0036 FFF7FEFF 		bl	HW_Select1_Read
 502              	.LVL79:
 503 003a 0028     		cmp	r0, #0
 504 003c E7D1     		bne	.L41
  37:main.c        ****         {
 505              		.loc 1 37 0 is_stmt 0 discriminator 1
 506 003e FFF7FEFF 		bl	HW_Select2_Read
 507              	.LVL80:
 508 0042 0128     		cmp	r0, #1
 509 0044 E3D1     		bne	.L41
  39:main.c        ****         }
 510              		.loc 1 39 0 is_stmt 1
 511 0046 FFF7FEFF 		bl	main_board
 512              	.LVL81:
 513 004a E0E7     		b	.L41
 514              		.cfi_endproc
 515              	.LFE33:
 516              		.size	main, .-main
 517              		.section	.rodata.str1.4,"aMS",%progbits,1
 518              		.align	2
ARM GAS  C:\Users\varun\AppData\Local\Temp\ccU3kTLK.s 			page 14


 519              	.LC0:
 520 0000 536D6172 		.ascii	"Smart_Box\000"
 520      745F426F 
 520      7800
 521 000a 0000     		.space	2
 522              	.LC2:
 523 000c 54657374 		.ascii	"Testing\000"
 523      696E6700 
 524              		.text
 525              	.Letext0:
 526              		.file 2 "Generated_Source\\PSoC4/LCD.h"
 527              		.file 3 "Generated_Source\\PSoC4/CyLib.h"
 528              		.file 4 "Generated_Source\\PSoC4/Status.h"
 529              		.file 5 "Generated_Source\\PSoC4/Router.h"
 530              		.file 6 "Generated_Source\\PSoC4/FAN.h"
 531              		.file 7 "Generated_Source\\PSoC4/SIC_1.h"
 532              		.file 8 "Generated_Source\\PSoC4/SOL_1.h"
 533              		.file 9 "Generated_Source\\PSoC4/SIC_2.h"
 534              		.file 10 "Generated_Source\\PSoC4/SOL_2.h"
 535              		.file 11 "Generated_Source\\PSoC4/SIC_3.h"
 536              		.file 12 "Generated_Source\\PSoC4/SOL_3.h"
 537              		.file 13 "Generated_Source\\PSoC4/SIC_4.h"
 538              		.file 14 "Generated_Source\\PSoC4/SOL_4.h"
 539              		.file 15 "Generated_Source\\PSoC4/SIC_5.h"
 540              		.file 16 "Generated_Source\\PSoC4/SOL_5.h"
 541              		.file 17 "Generated_Source\\PSoC4/SIC_6.h"
 542              		.file 18 "Generated_Source\\PSoC4/SOL_6.h"
 543              		.file 19 "Generated_Source\\PSoC4/SIC_7.h"
 544              		.file 20 "Generated_Source\\PSoC4/SOL_7.h"
 545              		.file 21 "Generated_Source\\PSoC4/SIC_8.h"
 546              		.file 22 "Generated_Source\\PSoC4/SOL_8.h"
 547              		.file 23 "Generated_Source\\PSoC4/HW_Select1.h"
 548              		.file 24 "Generated_Source\\PSoC4/HW_Select2.h"
